:100000000000000000005D28F100030EF20004086B
:10001000F3000A08F4008A01831203130B1F30282F
:10002000831603138C1E1928831203138C1E1928A0
:100030003B20831603130C1C3028831203130C1C63
:100040003028D003031D292851171430D000203048
:100050008506101051308E00C3308F0010140C1024
:100060008312031374088A0073088400720E8300DD
:10007000F10E710E09001819F81483177608840020
:100080001A08C4008000F60A8313981C4A28181224
:100090001816781544080E3C0318F815031856284E
:1000A00076081D3A031D0800F8155728080010307F
:1000B000F60083168C128312080083120313FC01CE
:1000C0008501860187018901F8011030F600903022
:1000D000F700831603138C309F003F3085000230F9
:1000E00086009830870000308900B101B201BD015F
:1000F000BE01831203138312031381309F008B010F
:1001000007148714071506119801981718168316F7
:1001100003139801181598161F30990083120313C2
:100120000B30F5003030900051308E00C3308F001E
:100130001430D000D1102D2491260615091000305E
:1001400048242D249F268618C1280030A60045305B
:10015000A5001630A4000630A3000430A20004302D
:10016000A1000930A0009030A7002D24F1242D24F7
:10017000CA252D241C30FA000030FB0014222D2447
:10018000A6261730FA000030FB0014222D24372257
:100190002D24D114D123FC231A242130A223423050
:1001A000A2235330A223C830A2237530A2230730E4
:1001B00040381D24003080381D248630A223831649
:1001C00003130C14831203138B170B170914F80174
:1001D000D114C401043086060000EF2500304038F9
:1001E0001D24003080381D249126F124831603132A
:1001F0008C16831203131816982698269826181220
:10020000831603138C1283120313440803194C2919
:1002100060304402031C0E292030C40244085530CB
:100220004406031D15293A234C2948304406031D72
:100230001C291030FC064C294B304406031D242990
:1002400075220430FC064C294C304406031D2C2931
:10025000C4260830FC064C2931304406031D3329DE
:100260002030FC064C2932304406031D3A29403028
:10027000FC064C2933304406031D41298030FC061E
:100280004C2945304406031D4C29F816DE22752200
:10029000F8120430FC064C2983120313C401D11454
:1002A0009F111F129F128326D11251128223D11641
:1002B0005112EA21013040381D241E3080381D249F
:1002C00075248326D11251129F151F129F12832667
:1002D0008223023040381D24183080381D24D1126A
:1002E0005112D113752483269F111F129F16832646
:1002F0008223033040381D24183080381D24D11249
:100300005116D1137524832651128316031337080F
:10031000B1003808B2000030B3000B30B4001C2626
:1003200083120313043040381D245F30B6000430BC
:1003300040381D24360880381D2400301F247526BF
:10034000B60B972983160313BB013C0883120313D2
:10035000003A0319B729B600043040381D24360886
:1003600080381D243C301F247526B60BAC2905307F
:1003700040381D24003080381D247530A22386307B
:10038000A223063040381D24183080381D24370839
:100390000523073040381D24003080381D24973055
:1003A000A223C426073040381D24183080381D246D
:1003B00038080523D1102E22472257226322FB2121
:1003C0003424F4217C0810390319E8293424372215
:1003D0002D24E828831603130310B10DB20DB10DBF
:1003E000B20D831203130800EB30A223F030A223D6
:1003F000370805230800EB30A223F530A223380884
:1004000005230800D1101B30FA000030FB00142235
:100410002D24D1140800D1101B30FA000030FB004D
:1004200014222D24D11408001B22FF3903190800BF
:100430003924FB0A142A831203177A088F007B08D9
:100440008D00831603178C170C1400000000831214
:10045000031700000C088312031308008312031310
:10046000C40120304124F124342434240800C40180
:100470002D241730FA005730FB0014222D247C1253
:100480000800C40145303924413039240800412294
:10049000D1125112313039243D3039249F111F12AD
:1004A0009F1283268223EA21D1165112712AD1127A
:1004B00051124122323039243D3039249F151F1208
:1004C0009F128326702AD1125116412233303924CB
:1004D0003D303924831203139F111F129F16832668
:1004E000822375243424C4010800053040381D24BB
:1004F000003080381D247530A223063040381D247A
:10050000183080381D2483171030F6008313F81E2E
:10051000AF22063040381D24183080381D24F901E0
:100520008030CA0083170F30F6008317F60A76086A
:1005300084000008831203138313C400AC00B023AB
:1005400031304406031DA62A4A08F9040310CA0CD8
:10055000031C952A7908B700B926C40108001A08B7
:100560007812F811C401831603138C168312031337
:10057000181644080319B92A1812831603138C128B
:1005800083120313F819D12A4408AC0041241B3A02
:10059000031978160319D52A44082C08B023F81D2E
:1005A000B22A83120313F811080083171030F600E3
:1005B0008313C40183120313F8110800831710304A
:1005C000F6008313831203131A087812F811C4017A
:1005D000831603138C168312031318164408031989
:1005E000EE2A1812831603138C1283120313F819C0
:1005F000FC2A83120313E72AC40183171030F60084
:10060000831383120313F8110800C400F900831642
:1006100003130830A200831203130310F90D031C07
:10062000303003183130AC00392483160313A20391
:1006300083120313031D0D2B3D30AC0039244408F5
:10064000F900790E0F39F63E0318073E3A3EAC002A
:1006500039248316031322088312031344080F3925
:10066000F63E0318073E3A3EAC0039246830AC0031
:1006700039240800D110B830A2232D24D11405301C
:1006800040381D24003080381D24A830A2230730B4
:1006900040381D24003080381D2483171030F600A8
:1006A000AF22073040381D24003080381D24781ACE
:1006B0000800CA0183171030F600831776088400FB
:1006C0000008F60A83120313C4000F30C405031098
:1006D000C40DC40DC40DC40D831776088400000832
:1006E000F60A831203130F394407C40083134A0820
:1006F000203E840044088000CA0ACA1D5D2BCA251A
:100700009F2608008312031300001F146E261F1576
:10071000D1131F19892B831203131E088316031389
:10072000B100B5001E08B200B60083120313832681
:10073000831603133508B7003608B8008312031375
:100740001F10080083120313B60036085624AC00AD
:10075000B60AFF39031908002C083924A52B080014
:100760008A11AD010A1600200A121F24AD0A0A16CA
:1007700000200A121F24AD0A0A1600200A121F24A4
:10078000AD0A0A1600200A121F24AD0A0A1600201C
:100790000A121F24AD0A0A1600200A121F24AD0AED
:1007A0000800DE235030B426E9235030B426EE236F
:1007B0005030B426FC235030B42608001330831682
:1007C0000313930000309400831203132830940025
:1007D000080007117C2607150000080021301D24A1
:1007E00090301D2405301D2413301D2420301D247D
:1007F0007C260C301D240800003014240030112405
:1008000008301D240930AA006030AB0000301F24DE
:10081000AB0B062CAA0B042C00301424003011243E
:10082000080080381D24080040381D2408000D30C1
:100830001D2408000C301D2408008710000007103C
:1008400093008C1D212C8C11000000000714000067
:1008500000008714000000000800831203130D300D
:1008600041240A3041240800831203130930412433
:10087000080083120313AC00D118B023D11C41240B
:1008800008008312031364000C1E442C9900080016
:1008900083120313B60036085624AC00B60AFF399B
:1008A000031908002C0839244B2C08008312031765
:1008B0008D00831603178C130C14831203170C0876
:1008C000831203130800640075080319712C0C1CB3
:1008D000712C1010F50B6D2C00340C100B308F00A8
:1008E00010148C1E632C1A08080083160313310899
:1008F000AF003208B0002F0EF038A500A507E23E89
:10090000A600323EA8002F080F39A607A607A807A1
:10091000E93EA700A707A707300E0F39A707A807CA
:10092000A70DA80DA809A80D30080F39A807A50D17
:100930000730A4000A30A807A703031C9B2CA707B5
:10094000A603031C9F2CA607A503031CA32CA50725
:10095000A403031CA72C83120313D11ED32C2B300A
:10096000D11B2D303924831603132508031DBD2CFC
:100970008312031320303924C12C83120313303E19
:100980003924831603132608303E39242E303924A7
:10099000831603132708303E3924831603132808CF
:1009A000303E39240800511EDA2C83160313240824
:1009B000303E3924831603132508303E392483162C
:1009C00003132608303E3924831603132708303ECC
:1009D0003924831603132808303E39242030392463
:1009E000080083120313220E0F39303E39242208E7
:1009F0000F39303E39242F303924210E0F39303E43
:100A0000392421080F39303E3924D1182030D11C27
:100A10002F303924D118142D200E0F39303E3924AF
:100A200020080F39303E392420303924240E0F3964
:100A3000031D1C2D20301D2D303E392424080F3974
:100A4000303E392448303924250E0F39303E3924C0
:100A500025080F39303E39244D303924260E0F3900
:100A6000303E392426080F39303E3924533039249A
:100A700008003A2D3B2D3C2D3D2D3E2D3F2D402D88
:100A8000412D422D432D442D452D462D472D482DDA
:100A9000492D4A2D4B2D4C2D4D2D080083168613C4
:100AA0008312861706173925861339250613080081
:100AB00083168613831286130617392586170800B6
:100AC00083168613831286133925061739250613D4
:100AD00008008316861383128617392506173925D1
:100AE0000613080083168617831239250617392541
:100AF0000315861B031106130800942539259D252F
:100B00003925080086178316031300008617831201
:100B10000313392508008316031386138312031366
:100B200000008613392508000617831603130000FA
:100B300006178312031339250800831603130613BF
:100B400083120313061339250800C7010830C900B2
:100B500082259425861FAD2DB02D0310C70DB42D11
:100B60000310C70DC70AB42D9D25C90BA92D080078
:100B7000C6000830C9000310C60D031CC02DC42DCB
:100B80008B257D258225C72D82257D25C72DC90B67
:100B9000BB2D080058258A264E25D030B825722551
:100BA000C5014508B82572252608B82572252508EF
:100BB000B82572252408B82572252308B825722582
:100BC0002208B82572252108B82572252008B825E5
:100BD00072259030B825692558258A2608005825A1
:100BE0006E264E25D030B8257225C5014508B8259A
:100BF0007225D1304E25D130B8256925A52560252F
:100C00004708A600A52560254708A500A52560255D
:100C10004708A400A52560254708A300A525602551
:100C20004708A200A52560254708A100A525602545
:100C30004708A000582508000310B901BA01103078
:100C4000A100B20DB10DBA0DB90D33083902031D63
:100C50002B2E34083A02031C332E3408BA02330810
:100C6000031CB30FB902BC0DBB0DA10B212E3B0819
:100C7000B1003C08B20008008316031303103408C7
:100C8000B2023308031C330FB102080065260310BB
:100C9000C00CBF0C031C522E3908BB070318BC0A3A
:100CA0003A08BC07BC0CBB0CBE0CBD0CC10B482EDB
:100CB000080042103908BB070318BC0A0318421485
:100CC0003A08BC074218031408001030C1003C0861
:100CD000C0003B08BF00BC01BB0108000130B300ED
:100CE0000130B4001430B500AD2E0130B300013036
:100CF000B4005030B500AD2E0130B3000430B40064
:100D00003230B500AD2E0130B3002030B400CC300D
:100D1000B500AD2E0130B3005030B4000130B50045
:100D2000AD2E0230B3007730B4000130B500AD2EE7
:100D30000430B3003130B4000130B500AD2E1030B6
:100D4000B3000E30B4003830B500AD2E2030B30003
:100D50002830B400DA30B500AD2EB50BAD2EB40B93
:100D6000AD2EB30BAD2E0800A9007C26A90BB52E25
:100D7000080058256E264E254830B82572253708BC
:100D8000B82569255825080058256E264E25483077
:100D9000013EB8257225A5254708B80069255825C4
:060DA000C4010800000080
:102000002C08B9000030BA00BC000630BB000A1230
:10201000462610308A001630B0003E088A073D0878
:102020002D0703188A0AB00703188A0A82070034AA
:102030000034003400340034003400340034003400
:1020400000340034003400340034003400340034F0
:1020500000340034003400340034003400340034E0
:1020600000340034003400340034003400340034D0
:1020700000340034003400340034003400340034C0
:1020800000340034003400340034003400340034B0
:1020900000340034003400340034003400340034A0
:1020A0000034003400340034003400340034003490
:1020B0000034003400340034003400340034003480
:1020C0000034003400340034003400340034003470
:1020D0000034003400340034003400340034003460
:1020E0000034003400340034003400340034003450
:1020F0000034003400340034003400340034003440
:10210000003400340034003400340034003400342F
:10211000003400340034003400340034003400341F
:10212000003400340034003400340034003400340F
:1021300000340034003400340034003400340034FF
:1021400000340034003400340034003400340034EF
:1021500000340034003400340034003400340034DF
:1021600000340034003400340034003400340034CF
:1021700000340034003400340034003400340034BF
:1021800000340034003400340034003400340034AF
:10219000003400340034003400340034003400349F
:1021A000003400340034003400340034003400348F
:1021B00000340034003400340034003400345F3420
:1021C0000034003400340034073400340734003461
:1021D000003414347F3414347F3414340034243401
:1021E0002A347F342A341234003426341634083426
:1021F0003434323400347634493455342234503453
:102200000034003400340534033400340034003426
:102210001C3422344134003400340034413422343C
:102220001C3400340034143408343E34083414347C
:102230000034083408343E340834083400340034A0
:102240005034303400340034003408340834083456
:10225000083408340034003460346034003400340E
:1022600000342034103408340434023400343E3452
:102270005134493445343E340034003442347F34E0
:1022800040340034003442346134513449344634EB
:1022900000342134413445344B3431340034183463
:1022A000143412347F341034003427344534453428
:1022B0004534393400343C344A34493449343034B8
:1022C00000340134013479340534033400343634B5
:1022D00049344934493436340034063449344934B5
:1022E00029341E340034003436343634003400349B
:1022F00000340034563436340034003400340034B2
:102300000834143422344134003414341434143472
:102310001434143400344134223414340834003476
:1023200000340234013451340934063400343E346C
:102330004134493455345E3400347E341134113420
:1023400011347E3400347F344934493449343634CE
:1023500000343E34413441344134223400347F343B
:102360004134413422341C3400347F3449344934FC
:102370004934413400347F34093409340934013498
:1023800000343E344134493449343A3400347F34E3
:102390000834083408347F340034003441347F3446
:1023A0004134003400342034413441343F3400346B
:1023B00000347F34083414342234413400347F3400
:1023C000403440344034403400347F3402340C34E0
:1023D00002347F3400347F340434083410347F34C2
:1023E00000343E344134413441343E3400347F348F
:1023F000093409340934063400343E34413451344C
:1024000021345E3400347F3409341934293446349D
:1024100000344634493449344934313400340134C9
:1024200001347F340134013400343F3440344034CB
:1024300040343F3400341F342034403420341F34BF
:1024400000343F3440343C3440343F34003463344F
:1024500014340834143463340034073408347034CA
:10246000083407340034613451344934453443343A
:10247000003400347F3441344134003400340234B9
:1024800004340834103420340034003441344134EE
:102490007F34003400340434023401340234043410
:1024A000003440344034403440344034003400344C
:1024B00001340234043400340034203454345434AD
:1024C0005434783400347F34483444344434383419
:1024D0000034383444344434443420340034383400
:1024E0004434443448347F3400343834543454341D
:1024F00054341834003408347E340934013402343E
:10250000003408345434543454343C3400347F346C
:1025100008340434043478340034003444347D34D2
:102520004034003400342034403444343D340034EA
:1025300000347F3410342834443400340034003400
:1025400041347F344034003400347C340434183453
:102550000434783400347C3408340434043478345B
:1025600000343834443444344434383400347C3413
:102570001434143414340834003408341434143447
:1025800018347C3400347C34083404340434083483
:102590000034483454345434543420340034043433
:1025A0003F3444344034203400343C3440344034EC
:1025B00020347C3400341C342034403420341C3427
:1025C00000343C344034383440343C3400344434F7
:1025D000283410342834443400340C34503450340B
:1025E00050343C3400344434643454344C34443433
:1025F00000340034083436344134003400340034BC
:1026000000347F3400340034003400344134363434
:10261000083400340034083408342A341C340834B4
:10262000003408341C342A340834083400340034AC
:1026300000340034003400340034003400340034FA
:1026400000340034003400340034003400340034EA
:1026500000340034003400340034003400340034DA
:1026600000340034003400340034003400340034CA
:1026700000340034003400340034003400340034BA
:1026800000340034003400340034003400340034AA
:10269000003400340034003400340034003400349A
:1026A000003400340034003400340034003400348A
:1026B000003400340034003400340034003400347A
:1026C000003400340034003400340034003400346A
:1026D000003400340034003400340034003400345A
:1026E000003400340034003400340034003400344A
:1026F000003400340034003400340034003400343A
:102700000034003400340034003400340034003429
:102710000034003400340034003400340034003419
:102720000034003400340034003400340034003409
:1027300000340034003400340034003400340034F9
:1027400000340034003400340034003400340034E9
:1027500000340034003400340034003400340034D9
:1027600000340034003400340034003400340034C9
:1027700000340034003400340034003400340034B9
:1027800000340034003400340034003400340034A9
:102790000034003400340034003400340034003499
:1027A0000034003400340034003400340034003489
:1027B00000340034003400340034003400345F341A
:1027C000003400340034003407340034073400345B
:1027D000003414347F3414347F34143400342434FB
:1027E0002A347F342A341234003426341634083420
:1027F000343432340034763449345534223450344D
:102800000034003400340534033400340034003420
:102810001C34223441340034003400344134223436
:102820001C3400340034143408343E340834143476
:102830000034083408343E3408340834003400349A
:102840005034303400340034003408340834083450
:102850000834083400340034603460340034003408
:1028600000342034103408340434023400343E344C
:102870005134493445343E340034003442347F34DA
:1028800040340034003442346134513449344634E5
:1028900000342134413445344B343134003418345D
:1028A000143412347F341034003427344534453422
:1028B0004534393400343C344A34493449343034B2
:1028C00000340134013479340534033400343634AF
:1028D00049344934493436340034063449344934AF
:1028E00029341E3400340034363436340034003495
:1028F00000340034563436340034003400340034AC
:10290000083414342234413400341434143414346C
:102910001434143400344134223414340834003470
:1029200000340234013451340934063400343E3466
:102930004134493455345E3400347E34113411341A
:1029400011347E3400347F344934493449343634C8
:1029500000343E34413441344134223400347F3435
:102960004134413422341C3400347F3449344934F6
:102970004934413400347F34093409340934013492
:1029800000343E344134493449343A3400347F34DD
:102990000834083408347F340034003441347F3440
:1029A0004134003400342034413441343F34003465
:1029B00000347F34083414342234413400347F34FA
:1029C000403440344034403400347F3402340C34DA
:1029D00002347F3400347F340434083410347F34BC
:1029E00000343E344134413441343E3400347F3489
:1029F000093409340934063400343E344134513446
:102A000021345E3400347F34093419342934463497
:102A100000344634493449344934313400340134C3
:102A200001347F340134013400343F3440344034C5
:102A300040343F3400341F342034403420341F34B9
:102A400000343F3440343C3440343F340034633449
:102A500014340834143463340034073408347034C4
:102A60000834073400346134513449344534433434
:102A7000003400347F3441344134003400340234B3
:102A800004340834103420340034003441344134E8
:102A90007F3400340034043402340134023404340A
:102AA0000034403440344034403440340034003446
:102AB00001340234043400340034203454345434A7
:102AC0005434783400347F34483444344434383413
:102AD00000343834443444344434203400343834FA
:102AE0004434443448347F34003438345434543417
:102AF00054341834003408347E3409340134023438
:102B0000003408345434543454343C3400347F3466
:102B100008340434043478340034003444347D34CC
:102B20004034003400342034403444343D340034E4
:102B300000347F34103428344434003400340034FA
:102B400041347F344034003400347C34043418344D
:102B50000434783400347C34083404340434783455
:102B600000343834443444344434383400347C340D
:102B70001434143414340834003408341434143441
:102B800018347C3400347C3408340434043408347D
:102B9000003448345434543454342034003404342D
:102BA0003F3444344034203400343C3440344034E6
:102BB00020347C3400341C342034403420341C3421
:102BC00000343C344034383440343C3400344434F1
:102BD000283410342834443400340C345034503405
:102BE00050343C3400344434643454344C3444342D
:102BF00000340034083436344134003400340034B6
:102C000000347F340034003400340034413436342E
:102C1000083400340034083408342A341C340834AE
:0E2C2000003408341C342A34083408340034DC
:102E00002034503449344334313436344634383441
:102E100037343734203461347634653463342034C5
:102E200062346F346F3474346C346F3461346434AE
:102E300065347234203451343D34313430344D34BF
:102E400068347A340A340D3420344D3450344C34E0
:102E50004134423420347634653472347334693406
:102E60006F346E34203438342E34313430340A34F4
:102E70000D3420344E344F344B34493441345F34B4
:102E80003834373437345F34583450344F34523454
:102E900054345F34303439343034373431343734A7
:102EA0002E34613473346D340A340D3400340A34F2
:102EB0000D343C3448343E3465346C3470340A3458
:102EC0000D343C3431343E3443346F346E34733417
:102ED000693467346E346534203431340A340D3447
:102EE0003C3432343E3443346F346E34733469349A
:102EF00067346E346534203432340A340D343C3453
:102F000033343E3443346F346E347334693467344D
:102F10006E346534203433340A340D343C344C344C
:102F20003E3465346334743475347234653420341B
:102F30005034433446340A340D343C3445343E3442
:102F400063347234693474347534723465342034C3
:102F50005034433446340A340D343C3455343E3412
:102F600070346434613474346534203452345434ED
:082F700043340A340D3400342F
:1036000020344C34453443345434553452344534E6
:1036100020344D3473346734203465346E342034B0
:1036200046344C34413453344834203464346534A3
:103630007034753469347334203430347834313430
:103640003834303430340A340D342034503461345A
:1036500067346534203420343D3420342034203421
:1036600020342034203420342034203420342034BA
:1036700020342034203420342034203420342034AA
:10368000203420342034203420340A340D342034C3
:103690005034613467346534203420343D34203470
:1036A000203420342034203420342034203420347A
:1036B000203420342034203420342034203420346A
:1036C00020342034203420342034203420340A3470
:1036D0000D34203450346134673465342034203460
:1036E0003D3420342034203420342034203420341D
:1036F000203420342034203420342034203420342A
:103700002034203420342034203420342034203419
:1037100020340A340D342034503461346734653435
:10372000203420343D3420342034203420342034DC
:1037300020342034203420342034203420342034E9
:1037400020342034203420342034203420342034D9
:103750002034203420340A340D3420345034613481
:1037600067346534203420343D3420342034203410
:1037700020342034203420342034203420342034A9
:103780002034203420342034203420342034203499
:10379000203420342034203420340A340D342034B2
:1037A00032343334343435343634373438343934CD
:1037B00030343134323433343434353436343734CD
:1037C00038343934303431343234333434343534B9
:1037D00036343734383439343034313432340A34CE
:0437E0000D34003470
:10380000203449346E34693474342034523454349E
:103810004334203470346134723420346434653479
:1038200066346134753474340A340D3420346134B0
:10383000753478342034763461346C3465347534BE
:1038400072347334203464346534663469346E34CD
:10385000693465347334203465346E342034643410
:103860007534723420342E342E340A340D3420341E
:10387000643461346E34733420346C3465342034F1
:10388000703472346F346734723461346D346D3433
:103890006534203463346134723420345234423419
:1038A00031343D34303420342E342E340A340D3447
:1038B00020342E342E342E342E342E342E342E3406
:1038C0002E342E342E342E342E342E342E342E34E8
:1038D0002E342E342E342E342E342E342E342E34D8
:1038E0002E342E342E342E342E342E342E340A34EC
:1038F0000D3420342E342E342E342E342E342E34E7
:103900002E342E342E342E342E342E342E342E34A7
:103910002E342E342E342E342E342E342E342E3497
:103920002E342E342E342E342E342E342E342E3487
:1039300020340A340D3420345634653472347334F0
:1039400069346F346E3420347334703465346334C6
:10395000693461346C3465342034583450344F3415
:10396000523454342E342E342E342E342E342E34FD
:103970002E342E3420340A340D342034323433348F
:1039800034343534363437343834393430343134EF
:1039900032343334343435343634373438343934DB
:1039A00030343134323433343434353436343734DB
:1039B000383439343034313432340A340D3400344C
:02400E00323D41
:104200003134363446343834373437342034773424
:10421000203462346F346F3474346C3464347234E8
:1042200051343D34313430344D3468347A342034B0
:1042300031343934323430343034623464347334A9
:104240000034303439342F3430343734203431347E
:1042500035344834323433344D34333432345334D7
:104260002034433448343034203420342034203453
:104270002034203420342034203475346E346934B2
:1042800074340034433448343134203420342034FE
:1042900020342034203450346F3469346E34743414
:1042A00073342034003443344834323420342034DE
:1042B0002034203420342034203450346F34693496
:1042C0006E34743473340034433448343534203419
:1042D0002034203420342034203450346F34693476
:1042E0006E34743473342034003450346F34723488
:1042F00074347334203438346234203450344334CA
:104300004634383435343734343400344534633447
:1043100072342034203420342034203420342034AB
:1043200020342034203420342034203400344C34E1
:104330006534633420342034203420342034203455
:1043400020342034203420342034203420340034ED
:104350004D3441344A3420344434533431343334CA
:104360003034373420342034203420342034203486
:10437000413441344D344D344A344A34573457343F
:10438000483448344D344D3453345334203420347D
:10439000203420342034203420342034203420347D
:1043A000203420342034203420342034203420346D
:1043B00000342E342E342E342E342E342E342E341B
:1043C0002E342E342E342E342E342E342E342E34DD
:1043D0002E342E34003450344334463420340034E8
:1043E0004534633472343D3400344C3465346334C2
:0443F0003D34003424
:00000001FF
